:020000040000FA
:0400000008EF1DF0F8
:08000800056ED8CF06F0E0CF31
:1000100007F00001E9CF0DF0EACF08F0E1CF09F0D9
:10002000E2CF0AF0D9CF0BF0DACF0CF0F3CF14F017
:10003000F4CF15F0FACF16F000C00FF001C010F0A9
:1000400002C011F003C012F004C013F0F2AA2CEFAA
:1000500000F0F2B428EF0BF0A0A232EF00F0A1B252
:10006000B2EF0BF0A0A438EF00F0A1B4AFEF09F0AD
:100070000FC000F010C001F011C002F012C003F078
:1000800013C004F00DC0E9FF08C0EAFF088E09C0E4
:10009000E1FF0AC0E2FF0BC0D9FF0CC0DAFF14C0B9
:1000A000F3FF15C0F4FF16C0FAFF055007C0E0FFCC
:1000B00006C0D8FF1000F76AC60FF66E000EF722D2
:1000C0000900F5501200000302FFFFFFFFFFFFFFD2
:1000D000FFFFFFFFFFFFF76AE60FF66E000EF72245
:1000E0000900F550120000FF02FFFFFFFFFFFFFFB6
:1000F000FFFFFFFFFFFFF76A060FF66E010EF72204
:100100000900F5501200080008004000000000003F
:1001100000000000000000000000000000000000DF
:1001200000000000000008AE03D0F2CF0EF0F29EF7
:10013000F76A480FF66E010EF7220900F55008AE77
:1001400002D00EBEF28E1200080000004000000037
:10015000000000000000000000000000000000009F
:100160000000000000000000F76A780FF66E010E34
:10017000F7220900F5501200090243000201008035
:1001800032090400000102020100052400100104EC
:10019000240202052406000105240100010705814F
:1001A000030800FA09040100020A00000007050222
:1001B000024000010705820240000100F76ACC0FEF
:1001C000F66E010EF7220900F55012000200F76AE0
:1001D000DE0FF66E010EF7220900F550120012171D
:1001E0001B20FFFFFFFFF76AF60FF66E010EF722E6
:1001F0000900F5501200120110010200000861040C
:100200003300000101020001F76A180FF66E020EBA
:10021000F7220900F5501200040309040803430003
:1002200043005300180353004500520049004100A9
:100230004C002000440045004D004F00F2CF0EF06E
:10024000F29EF76A560FF66E020EF7220900F5507D
:100250000EBEF28E1200280C0106F2CF0EF0F29EB6
:10026000F76A740FF66E020EF7220900F5500EBE03
:10027000F28E12000C444953504C41592076322ED4
:10028000300A6275696C642032202832332E313294
:100290002E3039290000F2CF0EF0F29EF76AB00F2F
:1002A000F66E020EF7220900F5500EBEF28E120015
:1002B0000C00F2CF0EF0F29EF76ACC0FF66E020E33
:1002C000F7220900F5500EBEF28E12003000F2CF78
:1002D0000EF0F29EF76AE80FF66E020EF7220900A2
:1002E000F5500EBEF28E12002E00F2CF0EF0F29EEE
:1002F000F76A040FF66E030EF7220900F5500EBEE2
:10030000F28E12000C4572723A00F2CF0EF0F29E9D
:10031000F76A240FF66E030EF7220900F5500EBEA1
:10032000F28E12002000F2CF0EF0F29EF76A400F1C
:10033000F66E030EF7220900F5500EBEF28E120083
:100340003A00F2CF0EF0F29EF76A5C0FF66E030EE3
:10035000F7220900F5500EBEF28E120020A86FBDE4
:100360000000F2CF0EF0F29EF76A7C0FF66E030EDD
:10037000F7220900F5500EBEF28E1200204269B33A
:100380000000F2CF0EF0F29EF76A9C0FF66E030E9D
:10039000F7220900F5500EBEF28E12002043657060
:1003A0000000F2CF0EF0F29EF76ABC0FF66E030E5D
:1003B000F7220900F5500EBEF28E120020AB65BF89
:1003C0000000F2CF0EF0F29EF76ADC0FF66E030E1D
:1003D000F7220900F5500EBEF28E120020A8BFBD14
:1003E0000000F2CF0EF0F29EF76AFC0FF66E030EDD
:1003F000F7220900F5500EBEF28E1200204379B2AA
:100400000000F2CF0EF0F29EF76A1C0FF66E040E9B
:10041000F7220900F5500EBEF28E1200204865E367
:100420000000F2CF0EF0F29EF76A3C0FF66E040E5B
:10043000F7220900F5500EBEF28E1200526F6F6D5A
:100440002000F2CF0EF0F29EF76A5C0FF66E040EFB
:10045000F7220900F5500EBEF28E12002B00F2CFEB
:100460000EF0F29EF76A780FF66E040EF72209007E
:10047000F5500EBEF28E120020200000F2CF0EF0DA
:10048000F29EF76A960FF66E040EF7220900F550F9
:100490000EBEF28E12002F00F2CF0EF0F29EF76A1F
:1004A000B20FF66E040EF7220900F5500EBEF28E62
:1004B0001200202020200000F2CF0EF0F29EF76AFA
:1004C000D20FF66E040EF7220900F5500EBEF28E22
:1004D00012004F5554202000F2CF0EF0F29EF76A22
:1004E000F20FF66E040EF7220900F5500EBEF28EE2
:1004F00012005365726765794B20444953504C4153
:1005000059320000F2CF0EF0F29EF76A1E0FF66E1F
:10051000050EF7220900F5500EBEF28E12000C31C6
:10052000772E5361766549440000F2CF0EF0F29EBB
:10053000F76A440FF66E050EF7220900F5500EBE5D
:10054000F28E12000C5772546F466C6173682D3E28
:100550000000F2CF0EF0F29EF76A6C0FF66E050EF9
:10056000F7220900F5500EBEF28E12004F4B00002C
:100570006492609462A402D06294FCD7BAEF09F04E
:10058000080E0201016F020E036F180E026F880E33
:10059000006F046B020E076F200E066F0001000C47
:1005A0000F0153A104D00001EBDF0F015391629AB8
:1005B0000001C3EF09F00F015F6B62920001C9EF08
:1005C00009F0036A0101CD51530FE96E0F0E0320AC
:1005D000EA6EEF6ACD51080DF350CF6BE96E020E53
:1005E000CF25EA6EEF6ACD51080DF350CF6BCE6F79
:1005F000040ECE27000ECF23CEC1E9FF020ECF2579
:10060000EA6EEF6A0001000C010E0101CC6FCC51C3
:10061000070807E3CCC1CDF10001D3DF0101CC2BEA
:10062000F6D70001000C2A6A296A250E286E800E72
:10063000276E2B6A2C6A080E2D6E7C6B7B912F6ABD
:100640002E6A776B7891000C0101C26BC2510108D0
:100650000AE3036AC251250FE96E000E0320EA6E19
:10066000EF6AC22BF3D70001DEDF1A6A010E1B6EA0
:10067000196A000C629600D000D000D0000C0F0167
:100680005F6B626A9F0E5B6F3D0E606E5C6B00017C
:10069000BBDFDADF160E0F01536F62A604D0000134
:1006A000E9DF0F01FAD7649800016ADF030E206EBC
:1006B000CFEF09F0608462986482D5EF09F0629C04
:1006C000DBEF09F0C7C121F0000CFF0E216E000C1A
:1006D0000101C56B245241E0C55107083EE31C509F
:1006E000000105E0020A0FE0010A19E024D0036AC4
:1006F0002350F2CFC7F1F29E37DD0101C7BFF28E62
:10070000C66F000118D0036A2350F2CFC7F1F29EE2
:100710007BDD0101C7BFF28EC66F00010CD0036AFA
:100720002350F2CFC7F1F29E5EDD0101C7BFF28E0A
:10073000C66F000100D0232A24060101C551C52B34
:10074000036A200F016E000E032201C0E9FF020EB2
:100750000324EA6EC6C1EFFFBDD7245204E1C551A0
:10076000080801E0196AC5C1C7F10001ABDF000C40
:10077000236A1C6A02011B51010A000107E0030AF7
:100780000AE0010A0BE0220A22E042D0120E246E97
:10079000030E1C6E3FD0430E246E3CD0020E1C6E26
:1007A000036A02011A511D0FE96E000E0320EA6E62
:1007B000EFCF23F0036A2350F2CFC4F1F29E000181
:1007C00023DD0101C4BFF28E246E000123D0036A31
:1007D00002011A51F2CFC4F1F29E0001F8DC0101CE
:1007E000C4BFF28E236E233C01D00FD0036A235086
:1007F000F2CFC4F1F29E0001B7DC0101C4BFF28E5A
:10080000246E000107D004D0010100015EDF0ED08C
:100810005CDF0CD002011F5305E124501E5D02E293
:100820001EC224F0010E196E000152DF5CEF05F0CC
:100830000101C45306E1040E206E0001E5DEE1D0A3
:100840000101050E206E020EC76F280EC66F010E45
:10085000C56FC5510708D8A0D4D0C5C1CDF10001DE
:10086000B0DE0101C86B036AC551F2CFCCF1F29E34
:10087000000131DC0101CCBFF28EFF085BE0040E09
:10088000C86FD890C535036AF2CFCCF1F29E000153
:100890004ADC0900F5CF03F00101CCBFF28EC96F2D
:1008A00003C0CAF1C551080DF350CD6BCC6F010EDA
:1008B000CC25016E000ECD21036E01C0E9FF020EB2
:1008C0000324EA6EC9C1EFFFC551080DF350CD6B8B
:1008D000CC6F020ECC25016E000ECD21036E01C03F
:1008E000E9FF020E0324EA6EC7C1ECFFED52C6C158
:1008F000EFFFD890C535036AF2CFCCF1F29E00012C
:1009000012DC0900F5CF03F00101CCBFF28EC6273F
:100910000350C723880ECB6FCAB1CB81CAB3CB8338
:10092000C551080DF350CD6BE96E020ECD25EA6E70
:10093000CBC1EFFF036AC551F2CFCCF1F29E0001AB
:100940005BEC00F00101CCBFF28EFF083CE0C883F5
:10095000C551080DF350CD6BCC6F040ECC27000EA3
:10096000CD23020ECC25016E000ECD21036E01C0F9
:10097000E9FF020E0324EA6EC7C1ECFFED52C6C1C7
:10098000EFFFD890C535036AF2CFCCF1F29E00019B
:100990007BEC00F00900F5CF03F00101CCBFF28E33
:1009A000C6270350C723C551080DF350CD6BCC6F3C
:1009B000040ECC27000ECD23CCC1E9FF020ECD25BD
:1009C000EA6E400EEF6EC851060802E10E0EC86FC7
:1009D000036AC551F2CFCCF1F29E00015BEC00F04E
:1009E0000101CCBFF28E0108D8A4C889036AC551A1
:1009F000530FE96E0F0E0320EA6EC8C1EFFFC52B3F
:100A000028D7000154EF05F00201195100010DE053
:100A1000010A15E0020A20E0060A2AE0030A31E092
:100A20000E0A30E0010A36E045D01BC020F2020178
:100A3000216B020E0101C76F000144DE3DD00201AF
:100A40001A2D07D0010E1B160101C76B00013ADEFB
:100A500002D000013ADE30D002011A2D06D01B82EE
:100A60000101C76B00012EDE02D000012EDE24D072
:100A7000020E196E1AC222F00101C76B000122DEBC
:100A80001BD076D61AC020F2010E0101C76F0001FB
:100A900019DE12D002011A5101080AE31AC21AF033
:100AA0001AC2C4F10001C4D60101C76B00010ADEFD
:100AB000000102D00ADE00D0FAEF06F01AC0C4F13D
:100AC00002011951000105E00A0A0CE0010A32E0B6
:100AD00046D00201206B216B020E0101C76F00019D
:100AE000F1DD3FD00101C45322E0010EC45D036A71
:100AF000F2CFC5F1F29E0001DEEC00F00101C5BFAE
:100B0000F28E016E02011C5DD8A002D001010FD04F
:100B1000036A1C51250FE96E000E0320EA6EEFCF29
:100B200020F2010E0101C76F0001CCDD02D00001EF
:100B3000CCDD17D00101C4530FE0036A02011C5140
:100B4000250FE96E000E0320EA6E1AC2EFFF0101C5
:100B5000C76B0001B7DD02D00001B7DD02D0B5DD03
:100B600000D0FAEF06F00101C591C4BFC581C49F52
:100B7000C5A113D0036AC451F2CFC6F1F29E0001A1
:100B80005BEC00F00101C6BFF28EFF0802E1000E2F
:100B900001D0010E016E13D012D0036AC451F2CFFE
:100BA000C6F1F29E00016BEC00F00101C6BFF28EAF
:100BB000FF0802E1000E01D0010E016E00D000011D
:100BC0005BEF06F00101C591C4BFC581C49FC5A1FB
:100BD00011D0C451080DF350C76BC66F040EC62761
:100BE000000EC723C6C1E9FF020EC725EA6E880EB4
:100BF000EF6E09D0C451080DF350C76BE96E020EB9
:100C0000C725EA6EEF6A00016AEF06F00101C5919F
:100C1000C4BFC581C49FC5A111D0C451080DF350F4
:100C2000C76BC66F040EC627000EC723C6C1E9FFF7
:100C3000020EC725EA6E840EEF6E0AD0C451080D6D
:100C4000F350C76BE96E020EC725EA6E840EEF6E95
:100C5000000172EF06F00101C591C4BFC581C49FB8
:100C6000C5A111D0C451080DF350C86BC76F040E55
:100C7000C727000EC823C7C1E9FF020EC825EA6EC8
:100C8000EFCFC6F10AD0C451080DF350C86BE96E1E
:100C9000020EC825EA6EEFCFC6F1C6AF02D0C6B5C8
:100CA00002D0000E01D0010E016E00017EEF06F0B1
:100CB0001CC2C4F158D701522EE002011951010A99
:100CC000000105E0020A0BE0030A11E022D01CC279
:100CD000C4F178D70101C76B0001F4DC1CD01CC241
:100CE000C4F194D70101C76B0001ECDC14D0020100
:100CF000206B216B1CC2C4F10001ADD7015203E08F
:100D0000010E0201206F020E0101C76F0001DADC43
:100D100002D0DBDC00D0FAEF06F0FE0E216E000CF4
:100D200002011C2D01D002D01C534EE119510001CB
:100D30000BE0010A0DE0210A1CE0010A1FE0030A92
:100D400030E0010A35E03DD0010E7E6FE6DF3BD09A
:100D5000020EEA6E200EE96EE26A300EE16E080EB7
:100D6000016EE6CFEEFF012EFCD71EC2C7F1AADC52
:100D70002AD0020E7E6F7B81D0DF25D0020EEA6E74
:100D8000200EE96EE26A270EE16E070E016EE6CFD5
:100D9000EEFF012EFCD7070E0101C76F000192DCA8
:100DA00012D01AC27CF00101C76B00018BDC0BD0A2
:100DB0001AC22FF01BC22EF00101C76B000182DCAA
:100DC00002D083DC00D002010001FAEF06F0196ABC
:100DD000020118517F0B000107E0010A06E0030A37
:100DE00005E0230A04E004D00FD668D661D798D76F
:100DF0006CDC00D006EF09F00101C451080DF3507E
:100E0000CA6BE96E020ECA25EA6EEFCFC6F1C55174
:100E1000020806E1C6AD02D0C56B02D0010EC56F57
:100E2000C551030813E1840EC66FC451080DF35079
:100E3000CA6BC96F040EC927000ECA23C9C1E9FFD6
:100E4000020ECA25EA6E840EEF6E07D0C52D03D0C0
:100E5000C80EC66F02D0880EC66FD890C435036A1C
:100E6000F2CFC9F1F29E000193EC00F00900F5CF3A
:100E700003F00101C9BFF28EC76F03C0C8F1C451AE
:100E8000080DF350CA6BC96F010EC925016E000E23
:100E9000CA21036E01C0E9FF020E0324EA6EC7C136
:100EA000EFFFC8B1C681C8B3C683C451080DF35063
:100EB000CA6BE96E020ECA25EA6EC6C1EFFF0001D9
:100EC000000C036A0101D251530FE96E0F0E03208B
:100ED000EA6EEF5212E0D251080DF350D46BD36F8B
:100EE000040ED327000ED423D3C1E9FF020ED4256C
:100EF000EA6EEFCFD3F1D3AF02D0000E01D0010ED6
:100F0000016E0001000CCDC1D2F1DBDF015264E0C3
:100F10000101CD51080DF350D36BD26F040ED227CF
:100F2000000ED323010ED225016E000ED321036ED5
:100F300001C0E9FF020E0324EA6ECEC1EFFFD051DB
:100F4000020817E1CD51080DF350D36BD26F040E98
:100F5000D227000ED323D2C1E9FF020ED325EA6EB9
:100F6000EFCFD1F1D1AD02D0D06B02D0010ED06F56
:100F700013D0D051040810E1CD51080DF350D36BBC
:100F8000E96E020ED325EA6EEFCFD1F1D1AD03D0D9
:100F9000010ED06F01D0D06BD02D03D0C80ED16F11
:100FA00002D0880ED16FCFB1D181CFB3D183CD51D3
:100FB000080DF350D36BD26F040ED227000ED3234B
:100FC000D2C1E9FF020ED325EA6ED1C1EFFF010EB7
:100FD000016E05D000D00001000E016E010100017C
:100FE000000C7E51010A05E0020A14E0010A19E032
:100FF0002CD0EA6A300EE96E020EE26E180EE16E37
:10100000080E016EE6CFEEFF012EFCD7030E7E6FB9
:1010100084DE1FD00101C76B000162EC03F07E6B20
:1010200018D0EA6A270EE96E020EE26E180EE16E23
:10103000070E016EE6CFEEFF012EFCD77E6B01019D
:10104000C76B000162EC03F004D07E6BC0EC02F0D1
:1010500000D054EF08F00101C551080DF350C76BE3
:10106000C66F010EC625016E000EC721036E01C0BA
:10107000E9FF020E0324EA6E036AEFCF01F003C01A
:1010800002F000014BEF08F078817A6B020E01014B
:10109000C56F0001E0D701C079F05BEF08F00101F6
:1010A000C45304E100019DD706D00101C4510208D8
:1010B00003E10001E9D701010001000CC5C15CFF9B
:1010C0000101C55303E0040E206E02D0020E206E13
:1010D000000170EF08F01A6A196A22C0C5F1EED754
:1010E000E0EF08F0C5C1D2F1ECDE015241E00101B0
:1010F000C551080DF350CE6BCD6F040ECD27000EF9
:10110000CE23020ECD25016E000ECE21036E01C04E
:10111000E9FF020E0324EA6EECCF03F0ED52EFCFAD
:10112000CBF103C0CCF1CCC1EAFFCBC1E9FFC7C111
:10113000E2FFC6C1E1FFC9C102F0C8C101F001521E
:1011400002E0022A02D0025206E0E6CFEEFF012EB4
:10115000FCD7022EFAD7C5C1CDF1C9C1CFF1C8C1A4
:10116000CEF1CAC1D0F10001CEDE015003D000D0D3
:10117000000E016E000C020E0101C56FC76B380E28
:10118000C66FC96B77C0C8F1020ECA6F0001AADF33
:1011900077C07DF0776B000C775301E0ECDFE7EF71
:1011A00008F00101C4530EE1192C05D0000168ECD0
:1011B00003F006D001011950020803E100018BD7AA
:1011C000010106D0C451020803E10001E5D7010185
:1011D0000001000C63300101C26FC233C2331F0E25
:1011E000C21763524EE1020100513C0B0101C36F73
:1011F000430E0201001700013AEC03F00101C35154
:10120000340822E10201046B0001E1D56498213C1D
:1012100007D00101C46B030EC56F0001EDDD12D0D4
:101220000101C46B020EC56F0001E6DD2150FE080E
:1012300009E00101CD6BCF6B21C0CEF1040ED06F60
:10124000000161DE1CD00101C351040819E1C46B27
:10125000000125DF0101C46B020EC56F0001CCDD6A
:101260002150FE080CE0213C01D009D00101CD6BDA
:10127000CF6B21C0CEF1010ED06F000144DE010121
:101280006BD0635004081DE1430E020104170001F6
:101290003AEC03F0FF0E216E0101C46B000181DF07
:1012A000213C01D00AD00101CD6BCF6B21C0CEF122
:1012B000020ED06F000127DE02D0C0EC02F04BD04E
:1012C000010163B41FD0C251080DF350C56B016E0C
:1012D000020EC525036EC251080DF350C76BE96EAF
:1012E000020EC725EA6EEF50430B03C0EAFF01C0B0
:1012F000E9FFEF6E00013AEC03F0C2C1C4F1CFDEAA
:101300002AD00101C251080DF350C56BC46F040E01
:10131000C427000EC523C4C101F0020EC525036E0B
:10132000C251080DF350C76BC66F040EC627000EDE
:10133000C723C6C1E9FF020EC725EA6EEF50430B73
:1013400003C0EAFFC4C1E9FFEF6E00013AEC03F00D
:10135000C2C1C4F126DF01010001E3EF09F0205210
:1013600001E13AD0625238E062A404D060A402D015
:10137000B8EF02F064A201D02FD062AA04D060AA14
:1013800002D0D0EF02F062A204D060A202D0DBEF64
:1013900002F062A004D060A002D03FEF03F062A888
:1013A00004D060A802D05AEF03F062AC04D060AC65
:1013B00002D05FEF03F00101C16B62A606D060A608
:1013C00004D0000107D702D0010105D00101C151AD
:1013D000C12B0308F2E20001A19438EF00F00101F3
:1013E000C751C919800BCB6FC7AF05D0C61FC71F28
:1013F000C62BD8B4C72BC9AF05D0C81FC91FC82B6F
:10140000D8B4C92B016A026A006A036AC95102E1B1
:10141000C85118E0100ECA6FD890C637C7370036CB
:101420000336C951035C02E1C851005C07E3C851AF
:10143000005ED8A00306C951035ED880013602368B
:10144000CA2FEAD7CBAF05D0011E021E012AD8B49D
:10145000022A0001000CBBC0C7F1BAC0C6F10101ED
:10146000C96B0A0EC86F0001BADF02C0C2F101C029
:10147000C1F1BDC0C7F1BCC0C6F10101C96B0A0E04
:10148000C86F0001ACDF02C0C4F101C0C3F1036A40
:1014900001019551600FE96E010E0320EA6EC1C192
:1014A000EFFF036A9551780FE96E010E0320EA6E93
:1014B000C3C1EFFF952B95511708D8A0956BC56B4D
:1014C000630E926F92C190F19D0E936F93C191F153
:1014D000C55117085EE3036AC551600FE96E010E3E
:1014E0000320EA6E9151800A006EEF50800A005C82
:1014F00009E2036AC551600FE96E010E0320EA6E2E
:10150000EFCF91F1036AC551780FE96E010E032008
:10151000EA6E9351800A006EEF50800A005C09E287
:10152000036AC551780FE96E010E0320EA6EEFCF12
:1015300093F1036AC551600FE96E010E0320EA6E54
:10154000EF50800A006E9051800A005C09E2036A45
:10155000C551600FE96E010E0320EA6EEFCF90F1E6
:10156000036AC551780FE96E010E0320EA6EEF5051
:10157000800A006E9251800A005C09E2036AC5513C
:10158000780FE96E010E0320EA6EEFCF92F1C52BC2
:101590009FD7000139EF0BF0F2CFC9F1F29EC7C11E
:1015A000A9FFA69CA69EA680A8500101C9BFF28EE5
:1015B000C85D16E0C7C1A9FFC8C1A8FFA69CA69E2A
:1015C000A684F250006EF29E0F01550EA76EAA0E71
:1015D000A76EA682A6B2FED7A6940050F212010111
:1015E0000001000C0101C16BC151170827E3036A18
:1015F000C151600FE96E010E0320EA6EEFCFC2F118
:10160000036AC151780FE96E010E0320EA6EEFCF35
:10161000C3F1D890C135200FC46F010EC425C56F2A
:10162000C4C1C7F1C2C1C8F10001B6DFC5C1C7F16D
:10163000C3C1C8F1B1DF0101C12BD6D7010EC52549
:10164000C66FC76F95C1C8F10001A6DF46EF0BF06A
:10165000872B87511008D8B07ED0862B876B865198
:101660003B08D8B076D0866B852B85513B080EE2BF
:10167000F2D6C80E0101C76FD3C0C8F100018CDFDC
:10168000842B856B8451090801E1ACD7845117087C
:10169000D8B05FD0832B846B83511C0802E3000E0B
:1016A00001D0010E0101C16F00018251020802E068
:1016B000000E01D0010E0101C11503E00001836B92
:1016C000822B000183511E0802E3000E01D0010E9F
:1016D0000101C16F00018251040802E0000E01D037
:1016E000010E0101C26F00018251060802E0000EE6
:1016F00001D0010E0101C21700018251040802E06D
:10170000000E01D0010E0101C2170001825109082B
:1017100002E0000E01D0010E0101C217000182514A
:101720000B0802E0000E01D0010E0101C215C11527
:1017300003E00001836B822B000183511F0802E24A
:10174000836B822B82510C0804E2802BD8B4812B4E
:10175000826BA92BB92BB051F908D8B0B02BF294F9
:1017600038EF00F0AA2BA19238EF00F0010EEA6EDC
:10177000B90EE96EEF5010E0030E016EBF0E006E61
:101780000400002EFDD7012EF9D7E30E006E002EC7
:10179000FED70400EF2EF0D7000C0101BDB102D03E
:1017A0008B9001D08B80BDB302D08B9201D08B8205
:1017B000BDB502D08B9401D08B84BDB702D08B967F
:1017C00001D08B8600008B88040000D000D0000080
:1017D0008B980001000C0101BE6B000E82B0010E5F
:1017E000BE13000E82B2010E006ED890003600507B
:1017F000BE13000E82B4010E006E00360036FC0EE1
:1018000000160050BE13000E82B6010E006E0036A8
:1018100000360036F80E00160050BE13BEC101F0AF
:101820000001000C94809482948494868B8E000036
:101830008B880000D0DF01C0BDF18B9800008B8841
:10184000040000D0C8DF01C0BCF18B989490949242
:10185000949494960101BD39006EF00E001600506C
:10186000BC11016E000137EF0CF08B9CDBD701C07F
:10187000BCF1010101AE02D00001F8D7BA5302E178
:101880008B9C01D08B8C00008B9E00008B98BB3909
:10189000BC6F0F0EBC17BCC1BDF100017EDF0101A2
:1018A000BB510F0BBC6FBD6F000177DF000C949034
:1018B0009492949494969498949C949E8B9C8B9ED2
:1018C0008B980F0E0101B96F000150DF010E01016D
:1018D0009B6F9B5103080CE3030EBD6F00015DDF9E
:1018E000050E0101B96F000141DF01019B2BF1D70A
:1018F000020EBD6F000151DF01019B6B9B5103087C
:1019000013E3036A9B51F2CF9CF1F29E00011EEC9F
:1019100001F001019CBFF28E9C6FBA6BBB6F00019E
:10192000A4DF01019B2BEAD7000148EF0DF0010174
:10193000BA6B400EBB6F000198DF04002C0E006EE6
:10194000002EFED7000001019B6B9B513F0818E35E
:10195000036A9B51D70FE96E000E0320EA6EEFCFAA
:101960009CF1010EBA6F9CC1BBF100017EDF040047
:10197000310E006E002EFED7000001019B2BE5D733
:10198000BA6B800EBB6F000170DF58EF0DF00101E4
:10199000B72D01D003D0400EB86F01D0B86B010E47
:1019A000B65DB827B8518009B96FBA6BBB6F00013B
:1019B0005CDF000C0101B5510C0A000105E0060ACC
:1019C0000FE0020A15E01BD00101BA6B010EBB6FDC
:1019D00000014BDF020E0101B96F0001C7DE17D015
:1019E000010E0101B66F020EB76F0001D0DF0FD0FC
:1019F0000101BA6B100EBB6F000137DF08D0010E7A
:101A00000101BA6FB5C1BBF100012FDF00D0000C9E
:101A1000646A606A616A925003090101926E206AE9
:101A2000186AF2BE188EF29E000124EC03F018BE74
:101A3000F28E1CEF0DF0ECD78DEF0DF0186AF2BEB0
:101A4000188EF29E24EC03F018BEF28E646A140E17
:101A5000616E606A6486010E206E000C070E816F55
:101A6000DA0E806F050E886F88C086F086C085F01C
:101A700085C084F084C083F083C082F0010E8A6F39
:101A80008B9AFF0E936EDF0E946E7E6A7F6A0FD77D
:101A9000F2CF9BF1F29EC80EA96EA69CA69EA680D0
:101AA000A85001019BBFF28E0001D46BD36F3FD7CA
:101AB000C69A010EC66E000EC76ED190800ED56E0E
:101AC000CD6A000ECA6E000ECB6EB16AB46A040015
:101AD000090E006E002EFED70000B450A19C8B9A18
:101AE0000C0EBD6EB76AB66A000E0409CA6E7F0E90
:101AF000CB6E010EBE6EF28A01019B6B9B51000101
:101B00002DEC01F0000908E001019B2BB56F0001ED
:101B100051DF0101F3D700018ED790DFFA0E0101EA
:101B2000B96F000123DEFA0E0101B96F00011EDE5C
:101B3000FA0E0101B96F000119DEFA0E0101B96F49
:101B4000000114DE01019A6B9A5118080AE3036A36
:101B50009A518D0FE96E000E0320EA6EEF6A9A2B00
:101B6000F3D7010E0001896FB26B8CEF1DF08A9ADA
:101B70009350DF0B0101936E0400F90E006E002EEE
:101B8000FED700000400E50E006E002EFED7000018
:101B900093502009936E04000E0E006E002EFED7A7
:101BA0000000A391A46BA4518B0804E3A42B81AA89
:101BB000A381F9D70400000EA3B1010E016E00014C
:101BC000000C9350DF0B0101936E040000D0935082
:101BD0002009936E04004F0E006E002EFED7000009
:101BE000000110EF0EF09350DF0B0101936E040023
:101BF0004F0E006E002EFED7000093502009936E0A
:101C0000000110EF0EF00101A56BA55107080DE3CF
:101C1000A451010B010802E10001D3D70001E3D771
:101C2000D8900101A433A52BF0D704000001000CCB
:101C30000101A36BA35107082CE3010E00017F6F84
:101C4000D8900101A5339350DF0B936E040000D0B0
:101C500093502009936E0400030E006E002EFED7F1
:101C6000000081BA03D000017F6B010181BA02D06C
:101C700000017F6B00017F2D03D00101A58F0001C2
:101C80000400310E006E002EFED700000101A32BD0
:101C9000D1D70400A5C101F00001000C0101A4513D
:101CA000A603F3CF01F0F4CF00F0A703F350002612
:101CB000A551A603F3500020026E0001000CF29C17
:101CC000F29EF2BEFDD7010E01019A6F9A510208F1
:101CD000D8A094D09A2D07D09C6BBBC09EF1BAC0FF
:101CE0009DF1BEC09FF19A51020808E1080E9C6F59
:101CF000BDC09EF1BCC09DF1BFC09FF1000137DFA8
:101D0000012C79D0040000D0550E0101A46F000110
:101D10007ADF0400630E006E002EFED70000010182
:101D20009B6B9B51070811E39C519B25036AC30FD2
:101D3000E96E000E0320EA6EEFCFA3F1A3C1A4F178
:101D4000000161DF01019B2BECD7BE0EA46F0001E7
:101D50005ADF0400630E006E002EFED7000068DF1D
:101D600001C0A0F165DF01C0A1F1A0C1D5F0A1C102
:101D7000D6F0D6C09EF1D5C09DF101019E31036E13
:101D80009D31026E033202320332023203320232DA
:101D90000F0E031602C09DF103C09EF1A151F00B7E
:101DA00002E0F00E9E13A0510F0BA26FA2510A0D7C
:101DB000F3CF00F00038A26F0F0EA2179EC1A5F15D
:101DC0009DC1A4F1A76B0A0EA66F000167DF010198
:101DD000A25101249D6F000E02209E6F9A2D04D007
:101DE0009EC1BBF09DC1BAF09A51020804E19EC1A8
:101DF000BDF09DC1BCF001019A2B68D70001B7DE90
:101E0000CC0E0101A46F0001FEDE040000D0440EE0
:101E10000101A46F0001F7DEC00EF212000C0101F7
:101E2000A091F2BEA081F29E000177513E0802E22D
:101E30003E0E776F7751772B036A380FE96E000EED
:101E40000320EA6E9FC1EFFFF29E0101A0B1F28E66
:101E5000186AF2BE188EF29E020ED26F000161EC7B
:101E600007F018BEF28E015208E0186AF2BE188E12
:101E7000F29EBBEC08F018BEF28E5CEF0FF07751CB
:101E80003E0817E2186AF2BE188EF29E020E010199
:101E9000D26F000161EC07F018BEF28E015208E02B
:101EA000186AF2BE188EF29EBBEC08F018BEF28ED5
:101EB000E6D79EC19FF1B3D7000C64B601D0BEDD5A
:101EC000202C0BD064BA09D0626A606AA084C00E6C
:101ED000F212110E606E020E206E000C020E010155
:101EE0009E6F0001CCDFE9DF9CC19EF1C8DF000CD2
:101EF00001019A6B9A5100014BEC01F0000907E0D7
:101F000001019A2BB56F000155DD0101F3D7200EB9
:101F100001019C6F0001E2DF000C01019B6B9B51F2
:101F200007081BE39B519A259D6FF2CF9EF1F29E0D
:101F30009DC1A9FFA69CA69EA680A8509EBFF28E1A
:101F40009C6F9B519A25036AC30FE96E000E032014
:101F5000EA6E9CC1EFFF9B2BE2D70001000C010150
:101F60009A6B0001DADF080E01019A6F0001D5DFDC
:101F700097EF1DF001019A6B9A5117082FE3D89043
:101F80009A35200F9B6F010E9B259C6F036A9A5117
:101F9000600FE96E010E0320EA6EF2CF9FF1F29E10
:101FA0009BC1A9FFA69CA69EA680A8509FBFF28EAB
:101FB000EF6E036A9A51780FE96E010E0320EA6E04
:101FC000F2CF9FF1F29E9CC1A9FFA69CA69EA6807F
:101FD000A8509FBFF28EEF6E9A2BCED7010E9C2594
:101FE0009D6FF2CF9EF1F29E9DC1A9FFA69CA69E79
:101FF000A680A8509EBFF28E956F000199EF1DF04C
:102000007891186AF2BE188EF29E020E0101C46F1A
:10201000C56F0001FCEC06F018BEF28E27EF10F041
:1020200078B101D0FDD77A517A2B036A300F016E57
:10203000000E032201C0E9FF020E0324EA6EEFCF77
:10204000B4F10101000179517A5D01E3D9D70101B1
:10205000B4C101F00001000C01019A51050803E12F
:1020600000018A6B01019A51060803E1010E00018B
:102070008A6F0001D5DF01C09BF19AC19CF12EDF70
:10208000ACEF1FF078B110D00101B451010805E3A5
:10209000B453D8B402D0000107D000010EDF040011
:1020A0000101B4070001EED7000CBADF01C0D5F082
:1020B000B7DF01C0D6F0D6C081F0D5C080F0150ED4
:1020C00001019C6F00010ADF88EF1EF001019B51A6
:1020D0003F0804E39BC19CF19D6B05D0400E9B5DC6
:1020E0009C6F010E9D6F010E9C259E6F010E9D251C
:1020F0009F6F9EC1B6F1B76F000149DC000CB2CFF3
:10210000D5F0B3CFD6F0D5C001F0D6C002F0000CA8
:102110000101BA6BBC6BBA510708D8A073D081BE5D
:1021200009D00001AA53D8B402D0010103D00400A1
:102130000101F5D781AE09D00001AA53D8B402D06D
:10214000010103D004000101F5D781BE09D00001CF
:10215000AA53D8B402D0010103D004000101F5D77D
:102160000001CDDF02C0BEF101C0BDF1AA510108DE
:1021700005E2030E0101966F45D00001AA6BB36A18
:10218000B26A0101BE51050804E305E1BD51DB0857
:1021900002E2000E01D0010EBF6FBE51220805E21F
:1021A000FF0A05E1BD51280802E3000E01D0010E2F
:1021B000BF110BE0040E966F010E0001AA6FBEC1A5
:1021C00098F1BDC197F101011DD0BE51130805E37F
:1021D00003E1BD51AF08D8B0BB6BBE51120810E28D
:1021E000FF0A03E1BD51CE080BE2010EBB6FBA51ED
:1021F000016E04E0D890BB37012EFCD7BB51BC1355
:10220000BA2B89D70001AF2D02D0BCC1ABF0AF51C2
:10221000020802E1BCC1ACF0AF51030802E1BCC14D
:10222000ADF0AF51040802E1BCC1AEF0BCC1B9F1E0
:10223000AA5304E1010E016E04D003D0000E016E1A
:1022400000D0000CB22D01D08AD0AF6BAFC096F198
:1022500096C1B4F1B4C1AEF0AEC0ADF0ADC0ACF05B
:10226000ACC0ABF0C00EF212850EB16EA082AA6BAC
:10227000B36AB26A81BE14D042DF02C0B8F101C0B5
:10228000B7F10101B8518B0808E2FF0A03E1B75129
:10229000A00803E2000104D0010104000001EAD714
:1022A0000101B8518B0808E2FF0A03E1B751A00809
:1022B00003E2010E966F4DD0B8512E0807E303E1FB
:1022C000B751DF0803E30A0E966F43D0020EB96FD1
:1022D0000001B6EC0BF0AA6BB36AB26A81AE04D00F
:1022E000AA5302E10400FAD7AA5305E0020E010145
:1022F000966F2FD00001AA6BB36AB26A010EAF6F5E
:10230000ABC0B9F105DF015203E1010122D00001A8
:10231000020EAF6FACC0B9F1FBDE015203E1010167
:1023200018D00001030EAF6FADC0B9F1F1DE01525C
:1023300003E101010ED00001040EAF6FAEC0B9F190
:10234000E7DE015203E1010104D00001A09207D0B1
:1023500001010001B26B000E016E05D004D0010E28
:10236000B26F016E00D0000C01019B6B9B511508F0
:102370000AE3036A9B519D0FE96E010E0320EA6E8A
:10238000EF6A9B2BF3D7FF0EB46F00017BDE78A1C1
:1023900004D046DE01C09AF102D001019A6B01011E
:1023A0009B6B9A531DE0036A9B519D0FE96E010ED2
:1023B0000320EA6E9AC1EFFFFF0EB46F000162DEE8
:1023C00078B103D001010CD000012ADE01C09AF1DE
:1023D00001019B2B9B51160801E202D00400E1D7BA
:1023E0009C6B9B519C5D27E2036A9C519D0FE96E9B
:1023F000010E0320EA6EEF5210E0036A9C519D0F1C
:10240000E96E010E0320EA6EEFCFB4F1B4C1B5F16D
:102410000001DAEC0CF00400010181BE03D00001E0
:1024200011DF010104009C510A0803E1000145DDB0
:1024300001019C2BD6D7000178A102D0F1DDFCD799
:10244000BCEF1EF001019A6B9A3D01D014D0F2CF7F
:102450009BF1F29E9AC1A9FFA69CA69EA680A850B9
:102460009BBFF28E9C6F9CC19EF1000108DD25DDB3
:1024700001019A2BE9D70001ACEF1FF001019A6B23
:102480009A3D01D015D0B46B0001FCDDC9DD01C05F
:102490009BF1186AF2BE188EF29E9AC1C7F101C074
:1024A000C8F1CCEC0AF018BEF28E01019A2BE8D7E5
:1024B0000001ACEF1FF0F29CF29EF2BEFDD7B7EC2C
:1024C0000DF0012C45D00400630E006E002EFED7E7
:1024D0000000330E0101A46F000103EC0EF00101B6
:1024E0009D6B9D51070830E3000118EC0EF001C010
:1024F0009EF101019D519C25036AC30FE96E000EF8
:102500000320EA6E9EC1EFFF9D519C259F6FA96E2F
:102510009EC1A8FFA69CA69EA684F2CF00F0F29EC4
:102520000F01550EA76EAA0EA76EA682A6B2FED701
:10253000A6940050F212010E0101B96F0001B6EC31
:102540000BF001019D2BCDD79D6BB46B00019ADD83
:10255000C00EF212000C01019B2D04D09C6B0001F7
:10256000AADF01019B51020805E1080E9C6F0001E2
:10257000A2DF01010001ACEF1FF0080E016E020E98
:10258000006E002EFED78A9C939C020E006E002ED9
:10259000FED70101A1378A98D8B09388D8A0939824
:1025A000938C81ACFED7012E01D002D00001E7D779
:1025B000020E006E002EFED78A9C939C000093882A
:1025C000020E006E002EFED7020E006E002EFED709
:1025D000938C81ACFED7016A020E006E002EFED7EE
:1025E00081B801808A9C939C8A9893980001000C82
:1025F0000101B46B000146DD13DD01503108D8A4A0
:102600008FD00101B46B00013DDD0ADD01503908B6
:10261000D8A47ED09388020E006E002EFED7938C35
:10262000020E006E002EFED78A989398020E006E5E
:10263000002EFED78A9C939CA20E0101A16F00017F
:102640009CDF01C09BF10400310E006E002EFED70E
:1026500000000101A16B000190DF0101A16B0001ED
:102660008CDF01019D6B9C6B9388020E006E002E27
:10267000FED7938C020E006E002EFED781ACFED7E3
:102680008A989398020E006E002EFED78A9C939C27
:10269000A20EA16F000171DF9DC19EF101019F6B30
:1026A0009DC1A1F1000169DF9CC1A1F166DF0101BB
:1026B000B46B0001E7DCB4DC01C09AF19AC1A1F16E
:1026C0005CDF01019A5305E19AC1A1F1000155DFD8
:1026D000010193980000938C81ACFED7020E006E2E
:1026E000002EFED700D000009388020E006E002E50
:1026F000FED7060EB96F0001B6EC0BF00400010125
:102700009C2BD8B49D2B9A5302E09A3DADD707D0AD
:10271000FF0E01019E6F00013FEC0FF0010107D099
:10272000FF0E01019E6F00013FEC0FF0010100015F
:1027300086EF1FF018C1EAFF17C1E9FF0101AFC121
:10274000EFFFE92AD8B4EA2AEF6A172BD8B4182B7E
:102750000001000CEACFAEF1E9CFADF10101A7AF66
:1027600008D0AD8FADA9AD2BA61FA71FA62BD8B43F
:10277000A72BA739F009A96FA927E20FAA6F320F7B
:10278000AC6FA7510F0BAA27AA27AC27E90FAB6F95
:10279000AB27AB27A6390F0BAB27AC27AB37AC3732
:1027A000AC1FAC37A6510F0BAC27A937070EA86F8B
:1027B0000A0EAB07AC27FDE3AA07AB27FDE3A90789
:1027C000AA27FDE3A807A927FDE3010EEA6EA80EDC
:1027D000E96E070EAD15AD9DE906AD1507E1ADB982
:1027E000E92AADB903D0200E006E1CD0E926AC0E4C
:1027F000E95CD8B4AD8DEF50006E08E1ADBD06D0F8
:10280000ADB91DD0ADB702D0200E0BD0ADAF06D004
:102810002D0E006EED50AD9DAD9F04D0AD87AD99EE
:10282000300E0026EACFA7F1E9CFA6F100C0AFF144
:10283000000180DFA7C1EAFFA6C1E9FF0101EE5058
:10284000ADADD5D70001000C01019D6B9E6B9F6B58
:10285000A06BA16BA26BA36BA46B010E186F9D0EF6
:10286000176F100EE96E9CC1A7F19BC1A6F1000184
:1028700071DF0101A56BA55107081CE3036AA5518F
:102880009D0FE96E010E0320EA6EEF5020080FE263
:10289000036AA5519D0FE96E010E0320EA6EEFCF8A
:1028A000A6F1A6C1B5F10001DAEC0CF00101A52BEF
:1028B0000400E1D70001000C01019B6B9B5100015A
:1028C00075EC01F0000908E001019B2BB56F0001D8
:1028D000DAEC0CF00101F2D701019C6B9AC19BF17B
:1028E0000001B2DFACEF1FF00101A951016AA85D40
:1028F00003E2A8C100F00CD0006A080EAA6FA83746
:102900000036A951005CD8B0006E0136AA2FF7D767
:102910000001000C016A026A006A036A0101A95100
:1029200002E1A85118E0100EAA6FD890A637A73779
:1029300000360336A951035C02E1A851005C07E3AD
:10294000A851005ED8A00306A951035ED8800136C5
:102950000236AA2FEAD70001000C0E0ED88082554D
:102960000101A36FA86F0C0EA96F0001BDDF01016B
:102970009D6B01C09CF19C510001805D01019E6F27
:102980009D510001815901019F6FA56B0C0EA46F31
:102990009DC1A7F19CC1A6F100014EEC0EF00150C3
:1029A00082250101A26F000E0220A36F020EA25D1C
:1029B000A06F000EA359A16F0001835101019E2554
:1029C000A26F000E9F21A36F9F31036E9E31026E96
:1029D000033202323F0E03160250A2270350A323F4
:1029E0009FC1A7F19EC1A6F1A96B640EA86F00015B
:1029F00091DF02C003F001500101A25F0250A35B0E
:102A00009FC1A7F19EC1A6F1010EA96F900EA86FFC
:102A1000000180DF02C003F001500101A227025033
:102A2000A323A56B1F0EA46FA1C1A7F1A0C1A6F19E
:102A300000014EEC0EF002C0A5F101C0A4F102C0ED
:102A4000A7F101C0A6F10101A96B0C0EA86F00014E
:102A500061DF02C003F001500101A225016EA35104
:102A600003220150580FA26F1B0E0320A36FA76F04
:102A7000A2C1A6F1A96B070EA86F00014BDF00C031
:102A800088F0882BD4EF15F0200E0101A3A9300E99
:102A9000A46FA2C100F0A2AF07D0001E002A00C0A0
:102AA000A2F12D0EA46FA38F0150A2C1A8F1640E54
:102AB000A96F000119DF00C0A2F1300E012401014D
:102AC000A56FA2C1A8F10A0EA96F00010DDF300E9B
:102AD00000240101A76F300E0124A66FA4C100F0ED
:102AE000A3A702D0A3AFA395A3B90BD0A3AF22D0C5
:102AF000A3B520D000C0A5F1A3B31CD000C0A6F19F
:102B000019D0300EA55D16E100C0A5F1200EA46F0E
:102B1000A3A704D0A395A383A3AFA393300EA65D70
:102B200009E100C0A6F1200EA56FA3A7F7D7A393D4
:102B3000A3AFA391A3A505D0A4C1AFF10001FADD15
:102B40000101A3A305D0A5C1AFF10001F3DD01018F
:102B5000A3A104D0A6C1AFF10001ECDDA7C1AFF184
:102B60000001E8DDBFEF15F0010E0101186F9F0EA7
:102B7000176F9EC1A2F1110EA36F000185D701014D
:102B80009F51200802E1300E9F6F300E9F5D006E56
:102B90000038A16FF00EA117300EA05DA127A1C1D2
:102BA00001F00001000CD9D69388020E006E002EB1
:102BB000FED7938C020E006E002EFED78A98939853
:102BC000020E006E002EFED78A9C939CD00E01014F
:102BD000A16F0001D2DC01C09BF10101A16B0001DA
:102BE000CCDC86C09EF1C0DF01C09AF19AC1A1F190
:102BF000C4DC85C09EF1B8DF01C09AF19AC1A1F191
:102C0000BCDC84C09EF1B0DF01C09AF19AC1A1F191
:102C1000B4DC88C0A1F1B1DC83C09EF1A5DF01C0A6
:102C20009AF19AC1A1F1A9DC82C09EF19DDF01C099
:102C30009AF19AC1A1F1A1DCD00E805D01019C6FD7
:102C4000070E0001815901019D6F9CC19EF1000199
:102C50008BDF01C09AF19AC1A1F18FDC01019A6B5F
:102C60009AC1A1F1000189DC93980000938C81AC9A
:102C7000FED7020E006E002EFED700D00000938813
:102C8000020E006E002EFED70400C0EF1FF00101FF
:102C90009C6B9D6B9E6B9F6BA06BA16BA26BA36BE0
:102CA000010E186F9C0E176F020EE96E9BC1A7F103
:102CB0009AC1A6F100014EDD0101A46BA4510708E1
:102CC00055E3036AA4519C0FE96E010E0320EA6EDE
:102CD000EF5020080FE2036AA4519C0FE96E010E29
:102CE0000320EA6EEFCFA6F1A6C1B5F10001DAEC40
:102CF0000CF00101A451020820E19BBF05D09B53B9
:102D00001CE19A51090819E39BAF08D09B51FE08BA
:102D100014E2FF0A03E19A51F6080FE2A66BA651EE
:102D2000000159EC01F0000909E00101A62BB56F83
:102D30000001DAEC0CF00101F2D700010101A4510D
:102D400002080FE1A66BA651000167EC01F0000933
:102D500009E00101A62BB56F0001DAEC0CF00101CE
:102D6000F2D700010101A42B0400A8D70001000C38
:102D7000080E0101A26F00C0A3F19388020E006E3D
:102D8000002EFED7938C81ACFED781B8D88081A865
:102D9000D8900136020E006E002EFED7939C8A9CBE
:102DA000A22FEBD79388020E006E002EFED78A98D2
:102DB000A351D8A493980000938C81ACFED7020E47
:102DC000006E002EFED78A9C939C020E006E002E91
:102DD000FED78A9893980001000C9388020E006E2B
:102DE000002EFED7938C020E006E002EFED78A981E
:102DF0009398020E006E002EFED78A9C939CD00EF4
:102E00000101A16F0001BDEC12F001C0A0F10101B0
:102E1000A16B0001BDEC12F09388020E006E002E33
:102E2000FED7938C020E006E002EFED781ACFED72B
:102E30008A989398020E006E002EFED78A9C939C6F
:102E4000D10E0101A16F0001BDEC12F0010E006E68
:102E50008FDF01507F0B01019F6F010E006E00019B
:102E600087DF01507F0B01019E6F010E006E000194
:102E70007FDF01503F0B01019D6F010E006E0001CD
:102E800077DF0150070B886F010E006E71DF015074
:102E90003F0B01019A6F010E006E000169DF0150C6
:102EA0001F0B01019B6F006A000162DF01C09CF1F2
:102EB00093980000938C81ACFED7020E006E002E1A
:102EC000FED700D000009388020E006E002EFED7C1
:102ED000040001019F517F0801E161D09F510F0B58
:102EE0000001866F01019F39006E0F0E0016005021
:102EF0000A0DF3500001862701019E510F0B0001BE
:102F0000856F01019E39006E0F0E001600500A0DEC
:102F1000F3500001852701019D510F0B0001846FC3
:102F200001019D39006E0F0E001600500A0DF3507E
:102F30000001842701019A510F0B0001836F0101E9
:102F40009A39006E0F0E001600500A0DF350000162
:102F5000832701019B510F0B0001826F01019B39F7
:102F6000006E0F0E001600500A0DF350000182276C
:102F700001019C510F0B0001806F816B01019C3995
:102F8000006E0F0E001600500A0DF350000180274E
:102F9000000E8123D00E8027070E8123010100013E
:102FA000A0EF1CF0BBC09CF1BAC09BF1BDC09EF16C
:102FB000BCC09DF101015E6B5D6B5EC15CF15DC1EA
:102FC0005BF15BC19AF19A510F0820E3D8909A35D2
:102FD000036A190FE96E010E0320EA6EECCF03F0CD
:102FE000ED52EF505B2703505C23D8909A35036A6B
:102FF000390FE96E010E0320EA6EECCF03F0ED52BB
:10300000EF505D2703505E239A2BDDD7186AF2BE7E
:10301000188EF29E5CC1C7F15BC1C6F1C96B100E80
:10302000C86F0001EFEC09F018BEF28E02C05CF12F
:1030300001C05BF1186AF2BE188EF29E5EC1C7F144
:103040005DC1C6F10101C96B100EC86F0001EFEC44
:1030500009F018BEF28E02C05EF101C05DF10101FF
:103060005CAF03D09CAF0AD002D09CBF09D05C51AA
:103070009C5D06E303E19B515B5D02E2D90E596F53
:103080009CAF03D05CAF0AD002D05CBF09D09C518A
:103090005C5D06E303E15B519B5D02E2DA0E596F72
:1030A0005B519B5D05E15C519C5D02E1430E596FF4
:1030B0005EAF03D09EAF0AD002D09EBF09D05E5152
:1030C0009E5D06E303E19D515D5D02E2D90E5A6FFC
:1030D0009EAF03D05EAF0AD002D05EBF09D09E5132
:1030E0005E5D06E303E15D519D5D02E2DA0E5A6F1B
:1030F0005D519D5D05E15E519E5D02E1430E5A6F9B
:10310000D8905F35036A190FE96E010E0320EA6E4D
:103110009CC1ECFFED529BC1EFFFD8905F35036A75
:10312000390FE96E010E0320EA6E9EC1ECFFED52ED
:103130009DC1EFFF5F2B5F510F08D8A05F6B0001AF
:10314000ABEF1CF001019B6BF29CF29EF2BEFDD72F
:1031500000018D5302E18C6B8B6B01019A6B9A51CC
:1031600017081AE3036A9A518D0F016E000E0322AD
:1031700003C09DF1010E9A25036A8D0FE96E000EC2
:103180000320EA6EEFCF9EF19DC1EAFF01C0E9FF87
:103190009EC1EFFF9A2BE3D70001A56B040001014C
:1031A0009A6B036A9A518D0FE96E000E0320EA6E46
:1031B000EF5205E09A51180802E39A2BF2D79A5180
:1031C0001308D8A002D10400590E006E002EFED7BD
:1031D00000009388020E006E002EFED7938C020E24
:1031E000006E002EFED78A989398020E006E002E75
:1031F000FED78A9C939CA30EA16F0001BDEC12F038
:1032000001019A511808D8A0C0D00400FE0E006E2B
:10321000002EFED7000004009A5117080FE3036A3E
:103220009A518D0FE96E000E0320EA6E010E006EBA
:1032300000019EDD01C0EFFF0DD00101036A9A512C
:103240008D0FE96E000E0320EA6E006A000190DD2A
:1032500001C0EFFF036A01019A518D0FE96E000E64
:103260000320EA6EEF3C02D09B2B01D09B6B9B515D
:10327000120809E2036A9A518D0FE96E000E0320CD
:10328000EA6EEF6A9B6B036A9A518D0FE96E000E2E
:103290000320EA6EEF52D8A471D0006A000168DD05
:1032A00093980000938C81ACFED7020E006E002E26
:1032B000FED700D000009388020E006E002EFED7CD
:1032C0009388020E006E002EFED7938C020E006EC5
:1032D000002EFED78A989398020E006E002EFED71D
:1032E0008A9C939CA20E0101A16F0001BDEC12F01B
:1032F0000101A16B0001BDEC12F00101A16B000105
:10330000BDEC12F09388020E006E002EFED7938C57
:10331000020E006E002EFED781ACFED78A989398DD
:10332000020E006E002EFED78A9C939CA30E010114
:10333000A16F0001BDEC12F001019A5117080FE3D3
:10334000036A9A518D0FE96E000E0320EA6E010E9A
:10335000006E00010DDD01C0EFFF0DD00101036A19
:103360009A518D0FE96E000E0320EA6E006A00018B
:10337000FFDC01C0EFFF8C6B8B6B01019A2B00010E
:103380008B2BD8B48C2B3CD7010193980000938CE5
:1033900081ACFED7020E006E002EFED700D00000DA
:1033A0009388020E006E002EFED793980000938C37
:1033B00081ACFED7020E006E002EFED700D00000BA
:1033C0009388020E006E002EFED79A6B010EB66F28
:1033D000020EB76F0001C7EC0CF001019A511308FF
:1033E0001BE3036A9A518D0FE96E000E0320EA6E0B
:1033F000EF520FE0036A9A518D0FE96E000E032021
:10340000EA6EEFCF9CF19CC1B5F10001DAEC0CF053
:1034100001019A2B0400E2D7C00EF2120001A62B84
:10342000D8B4A72BCCEF1CF078B183D28A2D81D2EF
:10343000A9510508D8B07DD2A96BA82D5DD0010E89
:103440000101B66FB76F0001C7EC0CF08451090899
:1034500010E301019A6B9A51000185EC01F000091B
:1034600008E001019A2BB56F0001DAEC0CF00101C4
:10347000F2D701019C6B84C09BF1000124EC14F095
:1034800001019A6B9A51000193EC01F0000909E0E7
:1034900001019A2BB56F0001DAEC0CF00101F2D7B3
:1034A00000018551090810E301019A6B9A5100014E
:1034B00059EC01F0000908E001019A2BB56F0001F9
:1034C000DAEC0CF00101F2D701019C6B85C09BF195
:1034D000000124EC14F001019A6B9A51000185EC73
:1034E00001F0000909E001019A2BB56F0001DAEC47
:1034F0000CF00101F2D70001A82DEFD0070E010159
:10350000B66F010EB76F0001C7EC0CF083510908CC
:1035100010E301019A6B9A51000159EC01F0000986
:1035200008E001019A2BB56F0001DAEC0CF0010103
:10353000F2D701019C6B83C09BF1000124EC14F0D5
:1035400001019A6B9A51000167EC01F0000909E052
:1035500001019A2BB56F0001DAEC0CF00101F2D7F2
:1035600000018251090810E301019A6B9A51000190
:1035700059EC01F0000908E001019A2BB56F000138
:10358000DAEC0CF00101F2D701019C6B82C09BF1D7
:10359000000124EC14F001019A6B9A51000167ECD0
:1035A00001F0000909E001019A2BB56F0001DAEC86
:1035B0000CF00101F2D7000181C09CF180C09BF1A9
:1035C00024EC14F08851020811E101019A6B9A5120
:1035D0000001A1EC01F0000909E001019A2BB56F8F
:1035E0000001DAEC0CF00101F2D700018851030868
:1035F00011E101019A6B9A510001B1EC01F000094F
:1036000009E001019A2BB56F0001DAEC0CF0010121
:10361000F2D700018851040811E101019A6B9A5117
:103620000001C1EC01F0000909E001019A2BB56F1E
:103630000001DAEC0CF00101F2D700018851050815
:1036400011E101019A6B9A510001D1EC01F00009DE
:1036500009E001019A2BB56F0001DAEC0CF00101D1
:10366000F2D700018851060811E101019A6B9A51C5
:103670000001E1EC01F0000909E001019A2BB56FAE
:103680000001DAEC0CF00101F2D7000188510708C3
:1036900011E101019A6B9A510001F1EC01F000096E
:1036A00009E001019A2BB56F0001DAEC0CF0010181
:1036B000F2D70001882D11D001019A6B9A510001B7
:1036C00001EC02F0000909E001019A2BB56F00013D
:1036D000DAEC0CF00101F2D70001A8510208D8A4DD
:1036E0008DD0010E0101B66FB76F0001C7EC0CF071
:1036F00001019A6B9A51000111EC02F0000909E0F6
:1037000001019A2BB56F0001DAEC0CF00101F2D740
:103710000001BBBF16D0BB5303E1BA51000811E250
:1037200001019A6B9A51000121EC02F0000909E0B5
:1037300001019A2BB56F0001DAEC0CF00101F2D710
:103740000001BBC09BF1BAC09AF147EC16F0040E21
:103750000101B56F0001DAEC0CF059C1B5F1DAECFA
:103760000CF001019A6B9A5100012FEC02F0000954
:1037700009E001019A2BB56F0001DAEC0CF00101B0
:10378000F2D700010E0E0101B66F010EB76F0001F6
:10379000C7EC0CF001019C6B90C19BF19BBF9C0797
:1037A000000124EC14F001019A6B9A5100013EECE7
:1037B00002F0000909E001019A2BB56F0001DAEC73
:1037C0000CF00101F2D7000101019C6B91C19BF14A
:1037D0009BBF9C07000124EC14F001019A6B9A51E5
:1037E00000014CEC02F0000909E001019A2BB56FD1
:1037F0000001DAEC0CF00101F2D70001A851030836
:10380000D8A48DD0010E0101B66FB76F0001C7ECCF
:103810000CF001019A6B9A5100015CEC02F0000976
:1038200009E001019A2BB56F0001DAEC0CF00101FF
:10383000F2D70001BDBF16D0BD5303E1BC51000853
:1038400011E201019A6B9A51000121EC02F000098A
:1038500009E001019A2BB56F0001DAEC0CF00101CF
:10386000F2D70001BDC09BF1BCC09AF147EC16F045
:10387000040E0101B56F0001DAEC0CF05AC1B5F18C
:10388000DAEC0CF001019A6B9A5100012FEC02F076
:10389000000909E001019A2BB56F0001DAEC0CF088
:1038A0000101F2D700010E0E0101B66F010EB76FD4
:1038B0000001C7EC0CF001019C6B92C19BF19BBF16
:1038C0009C07000124EC14F001019A6B9A5100014D
:1038D0003EEC02F0000909E001019A2BB56F0001EE
:1038E000DAEC0CF00101F2D7000101019C6B93C1ED
:1038F0009BF19BBF9C07000124EC14F001019A6B23
:103900009A5100014CEC02F0000909E001019A2BE8
:10391000B56F0001DAEC0CF00101F2D70001A82B21
:10392000A851030805E2010EA86FC22BB52BB62BD8
:1039300033D0A92D06D0B551070803E2EDEF16F0FC
:10394000B56BA951020808E1C251010805E25FEC1C
:103950000EF0D2EF17F0C26BA951030816E1B6536F
:1039600014E0D4C002F0D3C001F0023201320232BE
:103970000132023201C0BEFF02320230300B006E53
:10398000BD50CF0B0010BD6EB66BA951B85D04E001
:10399000A9C0B8F0A2EF18F0D1EF1FF0AB510208A8
:1039A00009E0AC51FD0806E0AC51030803E0AC515E
:1039B000FC082CE1FF0ED880AE55AD5D27E1AD517E
:1039C000B15D03E1B051060821E2030E01019E6FD3
:1039D00000013FEC0FF0AB51020803E0AC51FD08D1
:1039E00004E1ADC09EF13FEC0FF0AB51030803E0E2
:1039F000AC51FC0808E1E00EAD2501019A6F9E6F05
:103A000000013FEC0FF0B06BADC0B1F0DEEF1FF086
:103A1000F86AD09E088EEA6AE96AC150E00BC16E6E
:103A2000B46A1D6A040E1E6E0C0E1F6E206A246A94
:103A3000776B7E6B0A0EA96FB96BBA6BBB6BBC6BF5
:103A4000BD6BBE6BBF6BD36BD46B0E0ED76F110EFD
:103A5000D86F100ED96F1C0EDA6F100EDB6F110EBF
:103A6000DC6F0E0EDD6FDE6BDF6BE06BE16F100E57
:103A7000E26F1C0EE36F100EE46F0E0EE56FE66B47
:103A80000A0EE76FE86B040EE96FEA6FEB6FEC6FFD
:103A90000E0EED6FEE6B0A0EEF6FF06B0C0EF16F0A
:103AA000040EF26FF36FF46F0E0EF56FF66B020EED
:103AB000F76F050EF86F020EF96FFA6BFB6BFC6B7C
:103AC000FD6BFE6BFF6B0101006B1E0E016F080E9C
:103AD000026F040E036F080E046F1E0E056F066B57
:103AE0001F0E076F086B096F0A6B0B6F0C6B0D6F66
:103AF0000E6B0F6F106B116F126B136F146B156FD2
:103B0000166B176B5F6B906B916B926B936B946BF7
:103B1000956B00012EEF0DF00400C00EF2125FEC69
:103B20000EF0030EC26F78EC0FF0AFEF0FF0BAEFAC
:103B30000FF05DEC0FF078A105D010EC10F001C093
:103B400099F102D00101996B0101995100014BE0FB
:103B5000010A4AE0040A4FE0030A59E0010A5DE065
:103B60000D0AD8B468D01A0AD8B470D0010AD8B4F3
:103B70007DD0030AD8B48AD0010AD8B497D0070AF6
:103B8000D8B4A4D0210AD8B4B1D0200AD8B4BED0B9
:103B9000110AD8B4C3D0240AD8B4C9D0010AD8B401
:103BA000C9D0030AD8B4D2D0010AD8B4E3D0A30A4A
:103BB000D8B4EAD0010AD8B400D1030AD8B415D1D8
:103BC000010AD8B42AD1B20AD8B449D1070AD8B464
:103BD00069D1010AD8B468D10D0AD8B467D10A0AEC
:103BE000D8B481D1ABD1B8D1010E01019C6F0001D5
:103BF0006EEC0FF0B1D1FF0E01019E6F00013FECA2
:103C00000FF099C19EF13FEC0FF08A6BA5D1060E23
:103C100001019A6F00012CEF10F00101B46B00015B
:103C200042EC10F010EC10F0070E01019C6F000147
:103C30006EEC0FF091D1FF0E01019E6F00013FEC81
:103C40000FF099C19EF13FEC0FF086D110EC10F00F
:103C500001C084F0100E01019C6F00016EEC0FF0AA
:103C6000030E896FB46B89C0B3F076D110EC10F0FD
:103C700001C085F0110E01019C6F00016EEC0FF088
:103C8000030E896FB46B89C0B3F066D110EC10F0ED
:103C900001C086F0120E01019C6F00016EEC0FF066
:103CA000030E896FB46B89C0B3F056D110EC10F0DD
:103CB00001C083F0130E01019C6F00016EEC0FF048
:103CC000030E896FB46B89C0B3F046D110EC10F0CD
:103CD00001C082F0140E01019C6F00016EEC0FF028
:103CE000030E896FB46B89C0B3F036D110EC10F0BD
:103CF00001C088F0350E01019C6F00016EEC0FF0E1
:103D0000030E896FB46B89C0B3F026D155EF10F064
:103D1000030E896FB46B89C0B3F01ED1040E01018C
:103D20009C6F00016EEC0FF0010E8A6F15D178ECDC
:103D30000FF012D101019B6B000166EC10F0210E17
:103D400001019C6F00016EEC0FF006D10101B46B14
:103D5000000142EC10F010EC10F001C09AF101C02B
:103D60009BF166EC10F0220E01019C6F00016EECDD
:103D70000FF0F2D0B4EF11F0230E01019C6F00019F
:103D80006EEC0FF08A6BE8D0800E01019C6F000191
:103D90006EEC0FF0800E01019E6F00013FEC0FF002
:103DA000550E01019E6F00013FEC0FF0AA0E0101BC
:103DB0009E6F00013FEC0FF0CFD0810E01019C6F90
:103DC00000016EEC0FF0810E01019E6F00013FECCF
:103DD0000FF001019E6B00013FEC0FF0020E01019C
:103DE0009E6F00013FEC0FF0B7D0820E01019C6F77
:103DF00000016EEC0FF0820E01019E6F00013FEC9E
:103E00000FF0010E01019E6F00013FEC0FF0010168
:103E10009E6B00013FEC0FF09FD0830E01019C6F61
:103E200000016EEC0FF0830E01019E6F00013FEC6C
:103E30000FF001019A6B9A5100016CEC02F000093D
:103E400008E001019A2B9E6F00013FEC0FF0010189
:103E5000F2D701019E6B00013FEC0FF07DD0010114
:103E6000B46B000142EC10F010EC10F0D46B01C008
:103E7000D3F00101B46B000142EC10F010EC10F033
:103E800001019B6B01C09AF101C003F0000E00011B
:103E9000D3130150D413310E01019C6F00016EEC5D
:103EA0000FF05AD022EF12F03EEF12F001019A6BA0
:103EB0009A51000182EC02F0000908E001019A2BFE
:103EC000B56F0001DAEC0CF00101F2D70101B46B1F
:103ED000000142EC10F010EC10F001C09AF101C0AA
:103EE0009BF1ABEF12F001019A6B9A51000195EC36
:103EF00002F0000909E001019A2BB56F0001DAEC2C
:103F00000CF00101F2D70001F8EF12F0300E0101C0
:103F10009C6F00016EEC0FF001019A6B9A51000149
:103F2000A9EC02F0000909E001019A2BB56F00012C
:103F3000DAEC0CF00101F2D700010ED0FF0E010106
:103F40009E6F00013FEC0FF099C19EF13FEC0FF026
:103F500099C19AF15CEF14F004000101995302E059
:103F60000001B96B0001B951C80803E2B96B010E39
:103F70008A6F01019951120804E10001D3EF15F095
:103F8000010181BE04D0000122EC11F0010199531E
:103F900008E100018A2D01D002D0010102D014EF06
:103FA0001AF00001B22D0BD078B109D0010199535C
:103FB000D8B402D0000103D00001F0D4B26BB9D55F
:023FC0000300FC
:020000040030CA
:0E00000000C31E0E0000890003C000E0034094
:00000001FF
